:10F8000011241FBECFEFD0E1DEBFCDBF12E0A0E0DC
:10F81000B1E001C01D92A030B107E1F70E94327C37
:10F820000C941E7E0C94147C08955D9BFECF81E4A5
:10F830008CB95D9BFECF86E58CB95D9BFECF82E5E2
:10F840008CB95D9BFECF82E48CB95D9BFECF8FE4CB
:10F850008CB95D9BFECF8FE48CB95D9BFECF84E5B8
:10F860008CB908952F923F924F925F926F927F9240
:10F870008F929F92AF92BF92CF92DF92EF92FF92C0
:10F880000F931F93DF93CF9300D00F92CDB7DEB7C6
:10F8900004B603FE03C0E0E0F0E0099514BE88B3AF
:10F8A000806C88BB87B3806C87BBF894A89598E17F
:10F8B0000FB6F89491BD11BC0FBE8F98979A109215
:10F8C000900089E189B99AB986E080939500CC24AB
:10F8D000DD24EE24FF2400E21EE45F9B03C08CB114
:10F8E0008335A9F020E2C21623E0D20648F09798AB
:10F8F00088B38F7388BB87B38F7387BBF701099574
:10F900000894C11CD11CC8010197F1F7E6CF0E94F1
:10F91000157C1982AA24BB245F9BFECF9CB1913633
:10F9200021F45D9BFECF39E5A2C0913479F45F9B51
:10F93000FECF9CB15F9BFECF8CB15D9BFECF392E7D
:10F940002224A82EBB24A228B3280EC1923659F433
:10F950005D9BFECF89E58CB95D9BFECF91E09CB9A4
:10F960005D9BFECF19C1923409F086C05F9BFECF2C
:10F970009CB15F9BFECF8CB1592E4424C82EDD2450
:10F98000C428D5285F9BFECF3CB180E090E0E0E04A
:10F99000F1E08C159D0510F02FEF03C05F9BFECFAB
:10F9A0002CB12083019621E08030920711F031962E
:10F9B000F0CF6981663409F05CC0363409F039C093
:10F9C000750100E010E0EE0CFF1C001F111FA801E4
:10F9D0009701A0E0B1E08C9190E011969C90119776
:10F9E000882488299929129661E0F9010C01609315
:10F9F0006800E89511242E5F3F4F4F4F5F4F8EEF09
:10FA00009FEFC80ED91EC114D10429F765E0F70194
:10FA100060936800E8958091680080FDFCCF81E1EB
:10FA200080936800E8955695479537952795590135
:10FA30001BC03534C9F4DB82CA82850140E0E42E64
:10FA400041E0F42EF70161917F01C8010E94117E0F
:10FA50000F5F1F4F2A813B81215030403B832A8317
:10FA6000232B81F7AC0CBD1C5D9BFECF3DE03CB968
:10FA700053CF5D9BFECF90C0973609F047C05F9B88
:10FA8000FECF9CB15F9BFECF8CB1792E6624C82E31
:10FA9000DD24C628D7285F9BFECF8CB1863401F5C4
:10FAA000C501A0E0B0E0880F991FAA1FBB1FFC0191
:10FAB000259134915D9BFECF2CB95D9BFECF3CB967
:10FAC0000296A11DB11DEEEFFFEFCE0EDF1EC11499
:10FAD000D10469F7B695A795979587955C011CCFDA
:10FAE000853409F019CF76018501C8010E94097E8D
:10FAF0005D9BFECF8CB90F5F1F4F0894E108F108A2
:10FB0000E114F10491F7AC0CBD1C06CF9536D1F48D
:10FB1000F981F634A1F4E0E0F0E023E020936800FE
:10FB2000E8958091680080FDFCCFE050FF4F38EFF2
:10FB3000E030F30791F761E160936800E8955D9B21
:10FB4000FECF19C0953461F4E8E1F0E02CE00FB687
:10FB5000F894A895E1BD0FBE21BD5D9BFECF86CF79
:10FB6000903529F45D9BFECF6DE06CB9D5CE9C3409
:10FB700021F45D9BFECF8DE033C0903729F45D9B6F
:10FB8000FECF93E59CB9C8CE943741F45D9BFECF80
:10FB9000E6E4ECB95D9BFECF1CB8BECE892F88573A
:10FBA000823038F45F9BFECF8CB15D9BFECFFDE0D1
:10FBB00026C0943539F45F9BFECF2CB129835D9B21
:10FBC000FECF54CF933519F40E94157CA5CE9635FF
:10FBD00049F45D9BFECF60E36CB95D9BFECF88E38B
:10FBE0008CB99ACE933769F45D9BFECF92E09CB9B5
:10FBF0005D9BFECFE6E9ECB95D9BFECFFEE1FCB973
:10FC00008BCE9B3109F488CE5D9BFECF2FE32CB9C0
:10FC100083CEE199FECF9FBB8EBBE09A99278DB32F
:10FC20000895262FE199FECF9FBB8EBB2DBB0FB64B
:10FC3000F894E29AE19A0FBE01960895F894FFCFE6
:040000030000F80001
:00000001FF
